:020000040000FA
:100000008BEF03F0F76A140FF66E000EF72209006B
:10001000F550120053746570706572204D6F746FE7
:100020007220496E746572666163652076312C209A
:1000300062726F7567687420746F20796F752062C3
:10004000793A0A0D0000F76A560FF66E000EF72295
:100050000900F5501200416E647265772057696C93
:10006000736F6E0A0D00F76A760FF66E000EF722B8
:100070000900F55012007265636F6E6E73776F72D0
:100080006C642E636F6D0A0D0000F76A9A0FF66EAE
:10009000000EF7220900F550120052656164696E86
:1000A000672069733A2025346C753B20666F722097
:1000B000616E20617070726F78696D617465207611
:1000C0006F6C74616765206F663A202535660A0D8E
:1000D00000008E0E006E09C001F008C002F0036A35
:1000E000015209E102C001F0026A080E005E0152ED
:1000F00002E1006A08D0D89001BE04D00236013671
:100100000006F9D7019E0000DFEF03F00C50D8B4D1
:10011000A6D0186E1050D8B4A2D0185E01E205D057
:100120007F0E1826D8B09BD006D0810E185ED8A0BE
:1001300096D0D8B494D018C000F0016A026A036A5D
:10014000176A0DC016F0168E0EC015F00FC014F011
:10015000190E186E1350145E0DE2010E155E0AE2C0
:10016000165E08E2175E06E2172A162A152A1350B1
:10017000142628D01250155E12E2010E165E0FE210
:10018000175E0DE2172A162A125015261350142650
:1001900019E3152A17E1162A15E1172A13D0115071
:1001A0008009165E0EE2010E175E0BE2172A11504F
:1001B0008009162612501526E9E3162AE7E1172AC8
:1001C000E5D70380182E01D00BD0D8901436153601
:1001D00016361736D8900336023601361936BAD796
:1001E00019A006D0D890013202320332193202D05F
:1001F000000635E019BE1ED0D890143615361636D6
:1002000017361350145E07E2010E155E04E2165E07
:1002100002E2175E1AE31250155E05E2010E165E49
:1002200002E2175E12E311508009165E03E2010E2E
:10023000175E0BE3032A09E1022A07E1012A05E11F
:10024000002A0DE00132023203320DC018F01150C5
:10025000181A18AE02D0018E06D0019E04D0006A92
:10026000016A026A036A0000F6EF03F00C50D8B48A
:1002700071D0006E1050D8B46DD0002604E3810E0A
:10028000002668E204D07F0E005E64E363E00DC0E8
:1002900014F01150141A0D8E118E0F501302F4CF5A
:1002A00016F00E501202F4CF03F0F3CF15F0130244
:1002B000F3501626F4501522000E03220F5012029E
:1002C000F3501626F4501522000E026A0322022271
:1002D0000D501302F3501526F4500322000E022293
:1002E0000D501202F3500326F4500222000E016A50
:1002F00001220F501102F3501526F4500322000E74
:10030000022201220E501102F3500326F450022261
:10031000000E01220D501102F3500226F45001226A
:10032000002A01BE05D01536033602360136000616
:10033000000E15AE0AD0032A02220122015005E167
:10034000025003E1035001E1002A14BE018E14AEF5
:10035000019E04D0006A016A026A036A000005EF88
:1003600004F0EACF19F0E9CF18F01238F009146E52
:100370001426E20F156E320F176E12500F0B152652
:1003800015261726E90F166E1626162611380F0B9E
:100390001626172616361736171E173611500F0B4E
:1003A00017261436070E136E0A0E16061726FDE3DF
:1003B00015061626FDE314061526FDE3130614267E
:1003C000FDE3EA6A130EE96E070E1814E926170E0C
:1003D000E95C13E0EF50006E06E118B80CD018B6D7
:1003E00004D0200E03D0080E186E300E00260050E8
:1003F0009EA8FED7AD6EEE50EAD7EF50006E300EDD
:10040000002600509EA8FED7AD6E20EF04F016C067
:100410001FF017C020F0216A13AE02D01F8C2006F7
:10042000138E1250D8B49BD07F0E125C55E3126E1F
:10043000226A040E236ED8901536143613362136F0
:10044000232EF9D7040E125C08E2030E125CD8A426
:100450007CD00A0E215CD8A078D0030E125E222A2E
:100460003AD9D89015361436133621361FD9020ED4
:10047000236ED8902132133214321532232EF9D73D
:100480002AD9040E236ED890163217321832193238
:10049000232EF9D70BD91FD918C019F017C018F09F
:1004A00016C017F0166A02D916D917C019F016C06F
:1004B00018F0166A176AFAD821B6C4D7125205E1A5
:1004C000152A142A132A212A40D0D890153614361A
:1004D000133621361206B6D7121E122A7F0E1226A6
:1004E000226A040E236ED890153614361336213640
:1004F000232EF9D7040E1226050E125C32E3EBD838
:10050000D8901536143613362136D8901536143651
:1005100013362136CBD8D8901536143613362136FB
:10052000222A030E236ED890213213321432153250
:10053000232EF9D7030E125E21A8DED7D8902132E0
:100540001332143215321206D7D7121E122A030E96
:1005500012262228205ED8A0206A010E03D0020EA7
:1005600001D0000E1B6E1FBE0AD020BE08D0205244
:1005700006E0200E9EA8FED7AD6E202EFAD71FAC47
:1005800004D02D0E9EA8FED7AD6E1FAE0AD020BEA1
:1005900008D0205206E0300E9EA8FED7AD6E202E69
:1005A000F8D71F9E1F9C1BA007D022C01BF022C0A3
:1005B0001DF01F281D2628D01BA202D01F28226E46
:1005C0001F52D8B471D02E0E9EA8FED7AD6E22C099
:1005D0001EF01E061F501E5C02E31FC01EF01E52BE
:1005E00006E0300E9EA8FED7AD6E1E2EFAD722C0B2
:1005F00023F01F28235ED8B077D012061F281D6E67
:1006000022501D5E1DC01BF021C01AF0125005E0E3
:100610001C6ED8901A321C2EFCD71D5045E0300EAF
:100620001A249EA8FED7AD6E1B5006E11F523CE077
:100630002E0E9EA8FED7AD6E1B061D0635E012508D
:1006400005E01C6ED8901A361C2EFCD71A50215E7D
:1006500021C016F013C017F014C018F015C019F01F
:10066000D8901536143613362136D89015361436F0
:10067000133621361950152605E3142A03E1132AEF
:1006800001E1212A1850142603E3132A01E1212A4B
:1006900017501326D8B0212A16502126D890153687
:1006A000143613362136B0D700001ED01950152647
:1006B00005E3142A03E1132A01E1212A1850142624
:1006C00003E3132A01E1212A17501326D8B0212A67
:1006D00016502126000C21C016F013C017F014C0CC
:1006E00018F015C019F0000C00003CEF04F0EA6AA5
:1006F000080EE96EEF500DE0020E016E006A002E4A
:10070000FED7012EFBD7970E006E002EFED7EF2EE0
:10071000F3D747EF04F0F86AD09EEA6AE96AC1505D
:10072000C00B0309C16E070EB46EB450A19C700ECD
:10073000D36EB8960C0EAF6E220EAC6E900EAB6EF2
:10074000086A08505FDC082A006E00509EA8FED799
:10075000AD6E300E085CF5E1086A085074DC082ABA
:10076000006E00509EA8FED7AD6E0F0E085CF5E13E
:10077000086A085078DC082A006E00509EA8FED750
:10078000AD6E120E085CF5E1C150C00B0D09C16ED3
:10079000C050C00B0709C06EC09EC280040E016E1F
:1007A000C250C30B0110C26EC282C2B2FED7C45087
:1007B000076A066E07C009F006C008F08AD400C0B8
:1007C00008F001C009F002C00AF003C00BF003C03A
:1007D0000FF002C00EF001C00DF000C00CF0136A63
:1007E000126A7F0E116E860E106E90D40F6A0E6A1A
:1007F000200E0D6E810E0C6E03C013F002C012F0BD
:1008000001C011F000C010F031D500C00CF001C0E3
:100810000DF002C00EF003C00FF0106A105035DC6E
:10082000102A006E00509EA8FED7AD6E0C0E105C14
:10083000F5E1010EE96E07C012F006C011F091D586
:10084000100E116E115021DC112A006E00509EA86E
:10085000FED7AD6E310E115CF5E10FC015F00EC084
:1008600014F00DC013F00CC012F0196A186A010ED2
:10087000176E060E166ECBD50A0E9EA8FED7AD6E6D
:100880000D0E9EA8FED7AD6E640E086E30D7929006
:0A08900089708AD7010E016E030083
:020000040030CA
:0E00000000C90F1E008781000FC00FE00F40E7
:00000001FF
